 mlib_image

 Timestamp is 6710e056 (Thu Oct 17 10:00:54 2024)

 Preferred load address is 10000000

 Start         Length     Name                   Class
 0001:00000000 0007c25dH .text$mn                CODE
 0002:00000000 00000078H .idata$5                DATA
 0002:00000078 00000008H .00cfg                  DATA
 0002:00000080 00000004H .CRT$XCA                DATA
 0002:00000084 00000004H .CRT$XCZ                DATA
 0002:00000088 00000004H .CRT$XIA                DATA
 0002:0000008c 00000004H .CRT$XIZ                DATA
 0002:00000090 00000004H .CRT$XPA                DATA
 0002:00000094 00000004H .CRT$XPZ                DATA
 0002:00000098 00000004H .CRT$XTA                DATA
 0002:0000009c 00000004H .CRT$XTZ                DATA
 0002:000000a0 00000000H .gfids$y                DATA
 0002:000000a0 0000b520H .rdata                  DATA
 0002:0000b5c0 00000000H .rdata$CastGuardVftablesA DATA
 0002:0000b5c0 00000000H .rdata$CastGuardVftablesC DATA
 0002:0000b5c0 00000004H .rdata$sxdata           DATA
 0002:0000b5c4 00000074H .rdata$voltmd           DATA
 0002:0000b638 000002f4H .rdata$zzzdbg           DATA
 0002:0000b92c 00000004H .rtc$IAA                DATA
 0002:0000b930 00000004H .rtc$IZZ                DATA
 0002:0000b934 00000004H .rtc$TAA                DATA
 0002:0000b938 00000008H .rtc$TZZ                DATA
 0002:0000b940 00000090H .xdata$x                DATA
 0002:0000b9d0 00000124H .edata                  DATA
 0002:0000baf4 00000050H .idata$2                DATA
 0002:0000bb44 00000014H .idata$3                DATA
 0002:0000bb58 00000078H .idata$4                DATA
 0002:0000bbd0 0000028cH .idata$6                DATA
 0003:00000000 000002f8H .data                   DATA
 0003:000002f8 00000374H .bss                    DATA
 0004:00000000 00000060H .rsrc$01                DATA
 0004:00000060 00000328H .rsrc$02                DATA

  Address         Publics by Value              Rva+Base       Lib:Object

 0000:00000000       ___AbsoluteZero            00000000     <absolute>
 0000:00000000       ___arm64x_extra_rfe_table  00000000     <absolute>
 0000:00000000       ___arm64x_extra_rfe_table_size 00000000     <absolute>
 0000:00000000       ___arm64x_native_entrypoint 00000000     <absolute>
 0000:00000000       ___arm64x_redirection_metadata 00000000     <absolute>
 0000:00000000       ___arm64x_redirection_metadata_count 00000000     <absolute>
 0000:00000000       ___dynamic_value_reloc_table 00000000     <absolute>
 0000:00000000       ___enclave_config          00000000     <absolute>
 0000:00000000       ___guard_check_icall_a64n_fptr 00000000     <absolute>
 0000:00000000       ___guard_eh_cont_count     00000000     <absolute>
 0000:00000000       ___guard_eh_cont_table     00000000     <absolute>
 0000:00000000       ___guard_fids_count        00000000     <absolute>
 0000:00000000       ___guard_fids_table        00000000     <absolute>
 0000:00000000       ___guard_iat_count         00000000     <absolute>
 0000:00000000       ___guard_iat_table         00000000     <absolute>
 0000:00000000       ___guard_longjmp_count     00000000     <absolute>
 0000:00000000       ___guard_longjmp_table     00000000     <absolute>
 0000:00000000       ___hybrid_auxiliary_delayload_iat 00000000     <absolute>
 0000:00000000       ___hybrid_auxiliary_delayload_iat_copy 00000000     <absolute>
 0000:00000000       ___hybrid_auxiliary_iat    00000000     <absolute>
 0000:00000000       ___hybrid_auxiliary_iat_copy 00000000     <absolute>
 0000:00000000       ___hybrid_code_map         00000000     <absolute>
 0000:00000000       ___hybrid_code_map_count   00000000     <absolute>
 0000:00000000       ___hybrid_image_info_bitfield 00000000     <absolute>
 0000:00000000       ___x64_code_ranges_to_entry_points 00000000     <absolute>
 0000:00000000       ___x64_code_ranges_to_entry_points_count 00000000     <absolute>
 0000:00000001       ___safe_se_handler_count   00000001     <absolute>
 0000:00000100       ___guard_flags             00000100     <absolute>
 0000:00000000       ___ImageBase               10000000     <linker-defined>
 0001:00000000       _j2d_mlib_ImageAffine      10001000 f   mlib_ImageAffine.obj
 0001:00000050       _mlib_ImageAffine_alltypes 10001050 f   mlib_ImageAffine.obj
 0001:000003f0       _mlib_ImageAffineEdgeExtend_BC 100013f0 f   mlib_ImageAffineEdge.obj
 0001:00010530       _mlib_ImageAffineEdgeExtend_BL 10011530 f   mlib_ImageAffineEdge.obj
 0001:000159f0       _mlib_ImageAffineEdgeNearest 100169f0 f   mlib_ImageAffineEdge.obj
 0001:00016d60       _mlib_ImageAffineEdgeZero  10017d60 f   mlib_ImageAffineEdge.obj
 0001:00017630       _mlib_ImageAffine_d64_1ch_bc 10018630 f   mlib_ImageAffine_BC_D64.obj
 0001:00018100       _mlib_ImageAffine_d64_2ch_bc 10019100 f   mlib_ImageAffine_BC_D64.obj
 0001:00018cb0       _mlib_ImageAffine_d64_3ch_bc 10019cb0 f   mlib_ImageAffine_BC_D64.obj
 0001:00019870       _mlib_ImageAffine_d64_4ch_bc 1001a870 f   mlib_ImageAffine_BC_D64.obj
 0001:0001a420       _mlib_ImageAffine_f32_1ch_bc 1001b420 f   mlib_ImageAffine_BC_F32.obj
 0001:0001ae70       _mlib_ImageAffine_f32_2ch_bc 1001be70 f   mlib_ImageAffine_BC_F32.obj
 0001:0001b970       _mlib_ImageAffine_f32_3ch_bc 1001c970 f   mlib_ImageAffine_BC_F32.obj
 0001:0001c480       _mlib_ImageAffine_f32_4ch_bc 1001d480 f   mlib_ImageAffine_BC_F32.obj
 0001:0001cfa0       _mlib_ImageAffine_s32_1ch_bc 1001dfa0 f   mlib_ImageAffine_BC_S32.obj
 0001:0001db50       _mlib_ImageAffine_s32_2ch_bc 1001eb50 f   mlib_ImageAffine_BC_S32.obj
 0001:0001e7a0       _mlib_ImageAffine_s32_3ch_bc 1001f7a0 f   mlib_ImageAffine_BC_S32.obj
 0001:0001f400       _mlib_ImageAffine_s32_4ch_bc 10020400 f   mlib_ImageAffine_BC_S32.obj
 0001:00020050       _mlib_ImageAffine_d64_1ch_bl 10021050 f   mlib_ImageAffine_BL_D64.obj
 0001:000202f0       _mlib_ImageAffine_d64_2ch_bl 100212f0 f   mlib_ImageAffine_BL_D64.obj
 0001:00020690       _mlib_ImageAffine_d64_3ch_bl 10021690 f   mlib_ImageAffine_BL_D64.obj
 0001:00020b50       _mlib_ImageAffine_d64_4ch_bl 10021b50 f   mlib_ImageAffine_BL_D64.obj
 0001:00021150       _mlib_ImageAffine_f32_1ch_bl 10022150 f   mlib_ImageAffine_BL_F32.obj
 0001:000213f0       _mlib_ImageAffine_f32_2ch_bl 100223f0 f   mlib_ImageAffine_BL_F32.obj
 0001:00021790       _mlib_ImageAffine_f32_3ch_bl 10022790 f   mlib_ImageAffine_BL_F32.obj
 0001:00021c10       _mlib_ImageAffine_f32_4ch_bl 10022c10 f   mlib_ImageAffine_BL_F32.obj
 0001:000221a0       _mlib_ImageAffine_s32_1ch_bl 100231a0 f   mlib_ImageAffine_BL_S32.obj
 0001:000224b0       _mlib_ImageAffine_s32_2ch_bl 100234b0 f   mlib_ImageAffine_BL_S32.obj
 0001:00022900       _mlib_ImageAffine_s32_3ch_bl 10023900 f   mlib_ImageAffine_BL_S32.obj
 0001:00022ef0       _mlib_ImageAffine_s32_4ch_bl 10023ef0 f   mlib_ImageAffine_BL_S32.obj
 0001:00023660       _mlib_ImageAffine_d64_1ch_nn 10024660 f   mlib_ImageAffine_NN.obj
 0001:000237e0       _mlib_ImageAffine_d64_2ch_nn 100247e0 f   mlib_ImageAffine_NN.obj
 0001:00023990       _mlib_ImageAffine_d64_3ch_nn 10024990 f   mlib_ImageAffine_NN.obj
 0001:00023b60       _mlib_ImageAffine_d64_4ch_nn 10024b60 f   mlib_ImageAffine_NN.obj
 0001:00023d50       _mlib_ImageAffine_s32_1ch_nn 10024d50 f   mlib_ImageAffine_NN.obj
 0001:00023f90       _mlib_ImageAffine_s32_2ch_nn 10024f90 f   mlib_ImageAffine_NN.obj
 0001:00024130       _mlib_ImageAffine_s32_3ch_nn 10025130 f   mlib_ImageAffine_NN.obj
 0001:000242f0       _mlib_ImageAffine_s32_4ch_nn 100252f0 f   mlib_ImageAffine_NN.obj
 0001:000244d0       _mlib_ImageAffine_bit_1ch_nn 100254d0 f   mlib_ImageAffine_NN_Bit.obj
 0001:00024890       _mlib_ImageClippingMxN     10025890 f   mlib_ImageClipping.obj
 0001:00024ab0       _mlib_ImageColorTrue2IndexLine_S16_S16_3 10025ab0 f   mlib_ImageColorTrue2Index.obj
 0001:00027b20       _mlib_ImageColorTrue2IndexLine_S16_S16_4 10028b20 f   mlib_ImageColorTrue2Index.obj
 0001:0002cfc0       _mlib_ImageColorTrue2IndexLine_S16_U8_3 1002dfc0 f   mlib_ImageColorTrue2Index.obj
 0001:0002d390       _mlib_ImageColorTrue2IndexLine_S16_U8_4 1002e390 f   mlib_ImageColorTrue2Index.obj
 0001:0002d860       _mlib_ImageColorTrue2IndexLine_U8_S16_3 1002e860 f   mlib_ImageColorTrue2Index.obj
 0001:00030380       _mlib_ImageColorTrue2IndexLine_U8_S16_4 10031380 f   mlib_ImageColorTrue2Index.obj
 0001:000350b0       _mlib_ImageColorTrue2IndexLine_U8_U8_3 100360b0 f   mlib_ImageColorTrue2Index.obj
 0001:00035450       _mlib_ImageColorTrue2IndexLine_U8_U8_4 10036450 f   mlib_ImageColorTrue2Index.obj
 0001:00035940       _mlib_search_quadrant_S16_3 10036940 f   mlib_ImageColorTrue2Index.obj
 0001:00035a20       _mlib_search_quadrant_S16_4 10036a20 f   mlib_ImageColorTrue2Index.obj
 0001:00035b40       _mlib_search_quadrant_U8_3 10036b40 f   mlib_ImageColorTrue2Index.obj
 0001:00035c00       _mlib_search_quadrant_U8_4 10036c00 f   mlib_ImageColorTrue2Index.obj
 0001:00035d00       _mlib_search_quadrant_part_to_left_S16_3 10036d00 f   mlib_ImageColorTrue2Index.obj
 0001:00035f20       _mlib_search_quadrant_part_to_left_S16_4 10036f20 f   mlib_ImageColorTrue2Index.obj
 0001:000361a0       _mlib_search_quadrant_part_to_left_U8_3 100371a0 f   mlib_ImageColorTrue2Index.obj
 0001:00036380       _mlib_search_quadrant_part_to_left_U8_4 10037380 f   mlib_ImageColorTrue2Index.obj
 0001:000365b0       _mlib_search_quadrant_part_to_right_S16_3 100375b0 f   mlib_ImageColorTrue2Index.obj
 0001:000367e0       _mlib_search_quadrant_part_to_right_S16_4 100377e0 f   mlib_ImageColorTrue2Index.obj
 0001:00036a70       _mlib_search_quadrant_part_to_right_U8_3 10037a70 f   mlib_ImageColorTrue2Index.obj
 0001:00036c60       _mlib_search_quadrant_part_to_right_U8_4 10037c60 f   mlib_ImageColorTrue2Index.obj
 0001:00036e90       _mlib_ImageConvClearEdge_Bit 10037e90 f   mlib_ImageConvClearEdge_Bit.obj
 0001:000372e0       _mlib_ImageConvClearEdge_Fp 100382e0 f   mlib_ImageConvClearEdge_Fp.obj
 0001:00037710       _mlib_ImageConvCopyEdge_Bit 10038710 f   mlib_ImageConvCopyEdge_Bit.obj
 0001:00038480       _j2d_mlib_ImageConvKernelConvert 10039480 f   mlib_ImageConvKernelConvert.obj
 0001:00038df0       _j2d_mlib_ImageConvMxN     10039df0 f   mlib_ImageConvMxN.obj
 0001:00038e70       _mlib_ImageConvMxN_f       10039e70 f   mlib_ImageConvMxN.obj
 0001:00039800       _mlib_convMxNext_d64       1003a800 f   mlib_ImageConvMxN_Fp.obj
 0001:00039c00       _mlib_convMxNext_f32       1003ac00 f   mlib_ImageConvMxN_Fp.obj
 0001:00039ff0       _mlib_convMxNext_s32       1003aff0 f   mlib_ImageConvMxN_ext.obj
 0001:0003b490       _mlib_convMxNext_s16       1003c490 f   mlib_ImageConv_16ext.obj
 0001:0003d5b0       _mlib_i_convMxNext_s16     1003e5b0 f   mlib_ImageConv_16ext.obj
 0001:0003fa60       _mlib_convMxNnw_s16        10040a60 f   mlib_ImageConv_16nw.obj
 0001:00041720       _mlib_i_convMxNnw_s16      10042720 f   mlib_ImageConv_16nw.obj
 0001:00043440       _mlib_convMxNnw_s32        10044440 f   mlib_ImageConv_32nw.obj
 0001:00045ce0       _mlib_c_convMxNext_u8      10046ce0 f   mlib_ImageConv_8ext.obj
 0001:00047e20       _mlib_i_convMxNext_u8      10048e20 f   mlib_ImageConv_8ext.obj
 0001:0004a360       _mlib_c_convMxNnw_u8       1004b360 f   mlib_ImageConv_8nw.obj
 0001:0004c070       _mlib_i_convMxNnw_u8       1004d070 f   mlib_ImageConv_8nw.obj
 0001:0004db10       _mlib_convMxNnw_d64        1004eb10 f   mlib_ImageConv_D64nw.obj
 0001:0004f080       _mlib_convMxNnw_f32        10050080 f   mlib_ImageConv_F32nw.obj
 0001:00050e50       _mlib_convMxNext_u16       10051e50 f   mlib_ImageConv_u16ext.obj
 0001:00053040       _mlib_i_convMxNext_u16     10054040 f   mlib_ImageConv_u16ext.obj
 0001:00055510       _mlib_convMxNnw_u16        10056510 f   mlib_ImageConv_u16nw.obj
 0001:00057280       _mlib_i_convMxNnw_u16      10058280 f   mlib_ImageConv_u16nw.obj
 0001:00058710       _mlib_ImageCopy_bit_na     10059710 f   mlib_ImageCopy_Bit.obj
 0001:00058a90       _j2d_mlib_ImageCreate      10059a90 f   mlib_ImageCreate.obj
 0001:00058c30       _j2d_mlib_ImageCreateStruct 10059c30 f   mlib_ImageCreate.obj
 0001:00058c80       _j2d_mlib_ImageDelete      10059c80 f   mlib_ImageCreate.obj
 0001:00058cd0       _mlib_ImageSet             10059cd0 f   mlib_ImageCreate.obj
 0001:00058e60       _mlib_ImageSetSubimage     10059e60 f   mlib_ImageCreate.obj
 0001:00058f40       _mlib_ImageLookUpSI_S16_D64 10059f40 f   mlib_ImageLookUp_64.obj
 0001:00059200       _mlib_ImageLookUpSI_S32_D64 1005a200 f   mlib_ImageLookUp_64.obj
 0001:000594c0       _mlib_ImageLookUpSI_U16_D64 1005a4c0 f   mlib_ImageLookUp_64.obj
 0001:000596f0       _mlib_ImageLookUpSI_U8_D64 1005a6f0 f   mlib_ImageLookUp_64.obj
 0001:0005a0e0       _mlib_ImageLookUp_S16_D64  1005b0e0 f   mlib_ImageLookUp_64.obj
 0001:0005a400       _mlib_ImageLookUp_S32_D64  1005b400 f   mlib_ImageLookUp_64.obj
 0001:0005a710       _mlib_ImageLookUp_U16_D64  1005b710 f   mlib_ImageLookUp_64.obj
 0001:0005a9a0       _mlib_ImageLookUp_U8_D64   1005b9a0 f   mlib_ImageLookUp_64.obj
 0001:0005b4f0       _mlib_ImageLookUp_Bit_U8_1 1005c4f0 f   mlib_ImageLookUp_Bit.obj
 0001:0005b7e0       _mlib_ImageLookUp_Bit_U8_2 1005c7e0 f   mlib_ImageLookUp_Bit.obj
 0001:0005ba80       _mlib_ImageLookUp_Bit_U8_3 1005ca80 f   mlib_ImageLookUp_Bit.obj
 0001:0005bdc0       _mlib_ImageLookUp_Bit_U8_4 1005cdc0 f   mlib_ImageLookUp_Bit.obj
 0001:0005c1f0       _mlib_AffineEdges          1005d1f0 f   mlib_ImageScanPoly.obj
 0001:0005d790       _mlib_ilogb                1005e790 f   mlib_ImageUtils.obj
 0001:0005d800       _mlib_ImageAffineIndex_S16_S16_3CH_BC 1005e800 f   mlib_c_ImageAffineIndex_BC.obj
 0001:0005e6b0       _mlib_ImageAffineIndex_S16_S16_4CH_BC 1005f6b0 f   mlib_c_ImageAffineIndex_BC.obj
 0001:0005f920       _mlib_ImageAffineIndex_S16_U8_3CH_BC 10060920 f   mlib_c_ImageAffineIndex_BC.obj
 0001:000607b0       _mlib_ImageAffineIndex_S16_U8_4CH_BC 100617b0 f   mlib_c_ImageAffineIndex_BC.obj
 0001:000619f0       _mlib_ImageAffineIndex_U8_S16_3CH_BC 100629f0 f   mlib_c_ImageAffineIndex_BC.obj
 0001:000628a0       _mlib_ImageAffineIndex_U8_S16_4CH_BC 100638a0 f   mlib_c_ImageAffineIndex_BC.obj
 0001:00063b10       _mlib_ImageAffineIndex_U8_U8_3CH_BC 10064b10 f   mlib_c_ImageAffineIndex_BC.obj
 0001:000649a0       _mlib_ImageAffineIndex_U8_U8_4CH_BC 100659a0 f   mlib_c_ImageAffineIndex_BC.obj
 0001:00065be0       _mlib_ImageAffineIndex_U8_U8_3CH_BL 10066be0 f   mlib_c_ImageAffineIndex_BL.obj
 0001:00066190       _mlib_ImageAffineIndex_U8_S16_3CH_BL 10067190 f   mlib_c_ImageAffineIndex_BL.obj
 0001:00066720       _mlib_ImageAffineIndex_U8_U8_4CH_BL 10067720 f   mlib_c_ImageAffineIndex_BL.obj
 0001:00066e40       _mlib_ImageAffineIndex_U8_S16_4CH_BL 10067e40 f   mlib_c_ImageAffineIndex_BL.obj
 0001:00067530       _mlib_ImageAffineIndex_S16_U8_3CH_BL 10068530 f   mlib_c_ImageAffineIndex_BL.obj
 0001:00067ae0       _mlib_ImageAffineIndex_S16_S16_3CH_BL 10068ae0 f   mlib_c_ImageAffineIndex_BL.obj
 0001:00068070       _mlib_ImageAffineIndex_S16_U8_4CH_BL 10069070 f   mlib_c_ImageAffineIndex_BL.obj
 0001:00068790       _mlib_ImageAffineIndex_S16_S16_4CH_BL 10069790 f   mlib_c_ImageAffineIndex_BL.obj
 0001:00068e70       _mlib_ImageAffine_u8_1ch_bc 10069e70 f   mlib_c_ImageAffine_BC.obj
 0001:000692c0       _mlib_ImageAffine_u8_2ch_bc 1006a2c0 f   mlib_c_ImageAffine_BC.obj
 0001:000697b0       _mlib_ImageAffine_u8_3ch_bc 1006a7b0 f   mlib_c_ImageAffine_BC.obj
 0001:00069cb0       _mlib_ImageAffine_u8_4ch_bc 1006acb0 f   mlib_c_ImageAffine_BC.obj
 0001:0006a1a0       _mlib_ImageAffine_s16_1ch_bc 1006b1a0 f   mlib_c_ImageAffine_BC_S16.obj
 0001:0006a690       _mlib_ImageAffine_s16_2ch_bc 1006b690 f   mlib_c_ImageAffine_BC_S16.obj
 0001:0006ac30       _mlib_ImageAffine_s16_3ch_bc 1006bc30 f   mlib_c_ImageAffine_BC_S16.obj
 0001:0006b1d0       _mlib_ImageAffine_s16_4ch_bc 1006c1d0 f   mlib_c_ImageAffine_BC_S16.obj
 0001:0006b770       _mlib_ImageAffine_u16_1ch_bc 1006c770 f   mlib_c_ImageAffine_BC_U16.obj
 0001:0006bc60       _mlib_ImageAffine_u16_2ch_bc 1006cc60 f   mlib_c_ImageAffine_BC_U16.obj
 0001:0006c210       _mlib_ImageAffine_u16_3ch_bc 1006d210 f   mlib_c_ImageAffine_BC_U16.obj
 0001:0006c7c0       _mlib_ImageAffine_u16_4ch_bc 1006d7c0 f   mlib_c_ImageAffine_BC_U16.obj
 0001:0006cd70       _mlib_ImageAffine_u8_1ch_bl 1006dd70 f   mlib_c_ImageAffine_BL.obj
 0001:0006cfa0       _mlib_ImageAffine_u8_2ch_bl 1006dfa0 f   mlib_c_ImageAffine_BL.obj
 0001:0006d2c0       _mlib_ImageAffine_u8_3ch_bl 1006e2c0 f   mlib_c_ImageAffine_BL.obj
 0001:0006d6c0       _mlib_ImageAffine_u8_4ch_bl 1006e6c0 f   mlib_c_ImageAffine_BL.obj
 0001:0006dbe0       _mlib_ImageAffine_s16_1ch_bl 1006ebe0 f   mlib_c_ImageAffine_BL_S16.obj
 0001:0006de60       _mlib_ImageAffine_s16_2ch_bl 1006ee60 f   mlib_c_ImageAffine_BL_S16.obj
 0001:0006e1c0       _mlib_ImageAffine_s16_3ch_bl 1006f1c0 f   mlib_c_ImageAffine_BL_S16.obj
 0001:0006e610       _mlib_ImageAffine_s16_4ch_bl 1006f610 f   mlib_c_ImageAffine_BL_S16.obj
 0001:0006eb70       _mlib_ImageAffine_u16_1ch_bl 1006fb70 f   mlib_c_ImageAffine_BL_U16.obj
 0001:0006edf0       _mlib_ImageAffine_u16_2ch_bl 1006fdf0 f   mlib_c_ImageAffine_BL_U16.obj
 0001:0006f150       _mlib_ImageAffine_u16_3ch_bl 10070150 f   mlib_c_ImageAffine_BL_U16.obj
 0001:0006f5a0       _mlib_ImageAffine_u16_4ch_bl 100705a0 f   mlib_c_ImageAffine_BL_U16.obj
 0001:0006fb00       _mlib_ImageAffine_s16_1ch_nn 10070b00 f   mlib_c_ImageAffine_NN.obj
 0001:0006fc80       _mlib_ImageAffine_s16_2ch_nn 10070c80 f   mlib_c_ImageAffine_NN.obj
 0001:0006fe30       _mlib_ImageAffine_s16_3ch_nn 10070e30 f   mlib_c_ImageAffine_NN.obj
 0001:00070000       _mlib_ImageAffine_s16_4ch_nn 10071000 f   mlib_c_ImageAffine_NN.obj
 0001:00070200       _mlib_ImageAffine_u8_1ch_nn 10071200 f   mlib_c_ImageAffine_NN.obj
 0001:00070330       _mlib_ImageAffine_u8_2ch_nn 10071330 f   mlib_c_ImageAffine_NN.obj
 0001:000704e0       _mlib_ImageAffine_u8_3ch_nn 100714e0 f   mlib_c_ImageAffine_NN.obj
 0001:000706a0       _mlib_ImageAffine_u8_4ch_nn 100716a0 f   mlib_c_ImageAffine_NN.obj
 0001:00070880       _mlib_ImageConvClearEdge   10071880 f   mlib_c_ImageConvClearEdge.obj
 0001:00070e50       _mlib_ImageConvZeroEdge    10071e50 f   mlib_c_ImageConvClearEdge.obj
 0001:00070ee0       _mlib_ImageConvCopyEdge    10071ee0 f   mlib_c_ImageConvCopyEdge.obj
 0001:00072150       _mlib_ImageConvVersion     10073150 f   mlib_c_ImageConvVersion.obj
 0001:000721f0       _mlib_convMxNext_u8        100731f0 f   mlib_c_ImageConv_f.obj
 0001:00072250       _mlib_convMxNnw_u8         10073250 f   mlib_c_ImageConv_f.obj
 0001:000722b0       _mlib_ImageCopy_na         100732b0 f   mlib_c_ImageCopy.obj
 0001:00072450       _j2d_mlib_ImageLookUp      10073450 f   mlib_c_ImageLookUp.obj
 0001:00072ec0       _mlib_c_ImageLookUpSI_S16_S16 10073ec0 f   mlib_c_ImageLookUp_f.obj
 0001:00072ec0       _mlib_c_ImageLookUpSI_S16_U16 10073ec0 f   mlib_c_ImageLookUp_f.obj
 0001:000731a0       _mlib_c_ImageLookUpSI_S16_S32 100741a0 f   mlib_c_ImageLookUp_f.obj
 0001:00073460       _mlib_c_ImageLookUpSI_S16_U8 10074460 f   mlib_c_ImageLookUp_f.obj
 0001:00074170       _mlib_c_ImageLookUpSI_S32_S16 10075170 f   mlib_c_ImageLookUp_f.obj
 0001:00074170       _mlib_c_ImageLookUpSI_S32_U16 10075170 f   mlib_c_ImageLookUp_f.obj
 0001:00074440       _mlib_c_ImageLookUpSI_S32_S32 10075440 f   mlib_c_ImageLookUp_f.obj
 0001:00074700       _mlib_c_ImageLookUpSI_S32_U8 10075700 f   mlib_c_ImageLookUp_f.obj
 0001:00074970       _mlib_c_ImageLookUpSI_U16_S16 10075970 f   mlib_c_ImageLookUp_f.obj
 0001:00074970       _mlib_c_ImageLookUpSI_U16_U16 10075970 f   mlib_c_ImageLookUp_f.obj
 0001:00074bc0       _mlib_c_ImageLookUpSI_U16_S32 10075bc0 f   mlib_c_ImageLookUp_f.obj
 0001:00074e00       _mlib_c_ImageLookUpSI_U16_U8 10075e00 f   mlib_c_ImageLookUp_f.obj
 0001:000754e0       _mlib_c_ImageLookUpSI_U8_S16 100764e0 f   mlib_c_ImageLookUp_f.obj
 0001:00075e70       _mlib_c_ImageLookUpSI_U8_S32 10076e70 f   mlib_c_ImageLookUp_f.obj
 0001:00076810       _mlib_c_ImageLookUpSI_U8_U8 10077810 f   mlib_c_ImageLookUp_f.obj
 0001:000771d0       _mlib_c_ImageLookUp_S16_S16 100781d0 f   mlib_c_ImageLookUp_f.obj
 0001:000771d0       _mlib_c_ImageLookUp_S16_U16 100781d0 f   mlib_c_ImageLookUp_f.obj
 0001:000774b0       _mlib_c_ImageLookUp_S16_S32 100784b0 f   mlib_c_ImageLookUp_f.obj
 0001:000777b0       _mlib_c_ImageLookUp_S16_U8 100787b0 f   mlib_c_ImageLookUp_f.obj
 0001:00077a60       _mlib_c_ImageLookUp_S32_S16 10078a60 f   mlib_c_ImageLookUp_f.obj
 0001:00077a60       _mlib_c_ImageLookUp_S32_U16 10078a60 f   mlib_c_ImageLookUp_f.obj
 0001:00077d80       _mlib_c_ImageLookUp_S32_S32 10078d80 f   mlib_c_ImageLookUp_f.obj
 0001:000780c0       _mlib_c_ImageLookUp_S32_U8 100790c0 f   mlib_c_ImageLookUp_f.obj
 0001:00078360       _mlib_c_ImageLookUp_U16_S16 10079360 f   mlib_c_ImageLookUp_f.obj
 0001:00078360       _mlib_c_ImageLookUp_U16_U16 10079360 f   mlib_c_ImageLookUp_f.obj
 0001:000785c0       _mlib_c_ImageLookUp_U16_S32 100795c0 f   mlib_c_ImageLookUp_f.obj
 0001:00078840       _mlib_c_ImageLookUp_U16_U8 10079840 f   mlib_c_ImageLookUp_f.obj
 0001:00078a70       _mlib_c_ImageLookUp_U8_S16 10079a70 f   mlib_c_ImageLookUp_f.obj
 0001:00079b80       _mlib_c_ImageLookUp_U8_S32 1007ab80 f   mlib_c_ImageLookUp_f.obj
 0001:0007a600       _mlib_c_ImageLookUp_U8_U8  1007b600 f   mlib_c_ImageLookUp_f.obj
 0001:0007b4c0       _mlib_free                 1007c4c0 f   mlib_sys.obj
 0001:0007b4d0       _mlib_malloc               1007c4d0 f   mlib_sys.obj
 0001:0007b4d6       @__security_check_cookie@4 1007c4d6 f   MSVCRT:secchk.obj
 0001:0007b4f0       __alloca_probe             1007c4f0 f   MSVCRT:chkstk.obj
 0001:0007b4f0       __chkstk                   1007c4f0 f   MSVCRT:chkstk.obj
 0001:0007b51b       ___isa_available_init      1007c51b f   MSVCRT:cpu_disp.obj
 0001:0007b6f0       __allshl                   1007c6f0 f   MSVCRT:llshl.obj
 0001:0007b710       __aullshr                  1007c710 f   MSVCRT:ullshr.obj
 0001:0007ba6f       __DllMainCRTStartup@12     1007ca6f f   MSVCRT:dll_dllmain.obj
 0001:0007ba92       ___raise_securityfailure   1007ca92 f   MSVCRT:gs_report.obj
 0001:0007baba       ___report_gsfailure        1007caba f   MSVCRT:gs_report.obj
 0001:0007bc01       ___security_init_cookie    1007cc01 f   MSVCRT:gs_support.obj
 0001:0007bc4c       _DllMain@12                1007cc4c f   MSVCRT:dll_dllmain_stub.obj
 0001:0007bc6e       ?__scrt_initialize_type_info@@YAXXZ 1007cc6e f   MSVCRT:tncleanup.obj
 0001:0007bc7a       ?__scrt_uninitialize_type_info@@YAXXZ 1007cc7a f   MSVCRT:tncleanup.obj
 0001:0007bc86       ___local_stdio_printf_options 1007cc86 f i MSVCRT:default_local_stdio_options.obj
 0001:0007bc8c       ___local_stdio_scanf_options 1007cc8c f i MSVCRT:default_local_stdio_options.obj
 0001:0007bc92       ___scrt_initialize_default_local_stdio_options 1007cc92 f   MSVCRT:default_local_stdio_options.obj
 0001:0007bcf3       ___scrt_acquire_startup_lock 1007ccf3 f   MSVCRT:utility.obj
 0001:0007bd25       ___scrt_dllmain_after_initialize_c 1007cd25 f   MSVCRT:utility.obj
 0001:0007bd50       ___scrt_dllmain_before_initialize_c 1007cd50 f   MSVCRT:utility.obj
 0001:0007bd5e       ___scrt_dllmain_crt_thread_attach 1007cd5e f   MSVCRT:utility.obj
 0001:0007bd7d       ___scrt_dllmain_crt_thread_detach 1007cd7d f   MSVCRT:utility.obj
 0001:0007bd8a       ___scrt_dllmain_exception_filter 1007cd8a f   MSVCRT:utility.obj
 0001:0007bdbe       ___scrt_dllmain_uninitialize_c 1007cdbe f   MSVCRT:utility.obj
 0001:0007bde1       ___scrt_dllmain_uninitialize_critical 1007cde1 f   MSVCRT:utility.obj
 0001:0007bdee       ___scrt_initialize_crt     1007cdee f   MSVCRT:utility.obj
 0001:0007be27       ___scrt_initialize_onexit_tables 1007ce27 f   MSVCRT:utility.obj
 0001:0007beae       ___scrt_is_nonwritable_in_current_image 1007ceae f   MSVCRT:utility.obj
 0001:0007bf42       ___scrt_release_startup_lock 1007cf42 f   MSVCRT:utility.obj
 0001:0007bf5f       ___scrt_uninitialize_crt   1007cf5f f   MSVCRT:utility.obj
 0001:0007bf87       ___scrt_get_dyn_tls_init_callback 1007cf87 f   MSVCRT:dyn_tls_init.obj
 0001:0007bf8d       ___scrt_fastfail           1007cf8d f   MSVCRT:utility_desktop.obj
 0001:0007c0a8       __crt_debugger_hook        1007d0a8 f   MSVCRT:utility_desktop.obj
 0001:0007c0b0       __RTC_Initialize           1007d0b0 f   MSVCRT:initsect.obj
 0001:0007c0dc       __RTC_Terminate            1007d0dc f   MSVCRT:initsect.obj
 0001:0007c110       __SEH_prolog4              1007d110 f   MSVCRT:sehprolg4.obj
 0001:0007c155       __except_handler4          1007d155 f   MSVCRT:chandler4gs.obj
 0001:0007c184       @_guard_check_icall_nop@4  1007d184 f i MSVCRT:guard_support.obj
 0001:0007c187       __get_startup_argv_mode    1007d187 f   MSVCRT:argv_mode.obj
 0001:0007c18b       ___scrt_is_ucrt_dll_in_use 1007d18b f   MSVCRT:ucrt_detection.obj
 0001:0007c197       _memcpy                    1007d197 f   vcruntime:VCRUNTIME140.dll
 0001:0007c19d       _memset                    1007d19d f   vcruntime:VCRUNTIME140.dll
 0001:0007c1a3       ___std_type_info_destroy_list 1007d1a3 f   vcruntime:VCRUNTIME140.dll
 0001:0007c1a9       __except_handler4_common   1007d1a9 f   vcruntime:VCRUNTIME140.dll
 0001:0007c1af       __initterm                 1007d1af f   ucrt:api-ms-win-crt-runtime-l1-1-0.dll
 0001:0007c1b5       __initterm_e               1007d1b5 f   ucrt:api-ms-win-crt-runtime-l1-1-0.dll
 0001:0007c1bb       __seh_filter_dll           1007d1bb f   ucrt:api-ms-win-crt-runtime-l1-1-0.dll
 0001:0007c1c1       __configure_narrow_argv    1007d1c1 f   ucrt:api-ms-win-crt-runtime-l1-1-0.dll
 0001:0007c1c7       __initialize_narrow_environment 1007d1c7 f   ucrt:api-ms-win-crt-runtime-l1-1-0.dll
 0001:0007c1cd       __initialize_onexit_table  1007d1cd f   ucrt:api-ms-win-crt-runtime-l1-1-0.dll
 0001:0007c1d3       __execute_onexit_table     1007d1d3 f   ucrt:api-ms-win-crt-runtime-l1-1-0.dll
 0001:0007c1d9       __cexit                    1007d1d9 f   ucrt:api-ms-win-crt-runtime-l1-1-0.dll
 0001:0007c1df       ___acrt_initialize         1007d1df f   MSVCRT:ucrt_stubs.obj
 0001:0007c1df       ___acrt_thread_attach      1007d1df f   MSVCRT:ucrt_stubs.obj
 0001:0007c1df       ___acrt_thread_detach      1007d1df f   MSVCRT:ucrt_stubs.obj
 0001:0007c1df       ___acrt_uninitialize       1007d1df f   MSVCRT:ucrt_stubs.obj
 0001:0007c1df       ___acrt_uninitialize_critical 1007d1df f   MSVCRT:ucrt_stubs.obj
 0001:0007c1df       ___scrt_stub_for_acrt_initialize 1007d1df f   MSVCRT:ucrt_stubs.obj
 0001:0007c1df       ___scrt_stub_for_acrt_thread_attach 1007d1df f   MSVCRT:ucrt_stubs.obj
 0001:0007c1df       ___scrt_stub_for_acrt_thread_detach 1007d1df f   MSVCRT:ucrt_stubs.obj
 0001:0007c1df       ___scrt_stub_for_acrt_uninitialize 1007d1df f   MSVCRT:ucrt_stubs.obj
 0001:0007c1df       ___scrt_stub_for_acrt_uninitialize_critical 1007d1df f   MSVCRT:ucrt_stubs.obj
 0001:0007c1df       ___vcrt_initialize         1007d1df f   MSVCRT:ucrt_stubs.obj
 0001:0007c1df       ___vcrt_thread_attach      1007d1df f   MSVCRT:ucrt_stubs.obj
 0001:0007c1df       ___vcrt_thread_detach      1007d1df f   MSVCRT:ucrt_stubs.obj
 0001:0007c1df       ___vcrt_uninitialize       1007d1df f   MSVCRT:ucrt_stubs.obj
 0001:0007c1df       ___vcrt_uninitialize_critical 1007d1df f   MSVCRT:ucrt_stubs.obj
 0001:0007c1e2       ___scrt_stub_for_is_c_termination_complete 1007d1e2 f   MSVCRT:ucrt_stubs.obj
 0001:0007c1e2       __is_c_termination_complete 1007d1e2 f   MSVCRT:ucrt_stubs.obj
 0001:0007c1e5       __filter_x86_sse2_floating_point_exception 1007d1e5 f   MSVCRT:x86_exception_filter.obj
 0001:0007c1e5       __filter_x86_sse2_floating_point_exception_default 1007d1e5 f   MSVCRT:x86_exception_filter.obj
 0002:00000000       __imp__IsProcessorFeaturePresent@4 1007e000     kernel32:KERNEL32.dll
 0002:00000004       __imp__UnhandledExceptionFilter@4 1007e004     kernel32:KERNEL32.dll
 0002:00000008       __imp__SetUnhandledExceptionFilter@4 1007e008     kernel32:KERNEL32.dll
 0002:0000000c       __imp__GetCurrentProcess@0 1007e00c     kernel32:KERNEL32.dll
 0002:00000010       __imp__TerminateProcess@8  1007e010     kernel32:KERNEL32.dll
 0002:00000014       __imp__QueryPerformanceCounter@4 1007e014     kernel32:KERNEL32.dll
 0002:00000018       __imp__GetCurrentProcessId@0 1007e018     kernel32:KERNEL32.dll
 0002:0000001c       __imp__GetCurrentThreadId@0 1007e01c     kernel32:KERNEL32.dll
 0002:00000020       __imp__GetSystemTimeAsFileTime@4 1007e020     kernel32:KERNEL32.dll
 0002:00000024       __imp__DisableThreadLibraryCalls@4 1007e024     kernel32:KERNEL32.dll
 0002:00000028       __imp__InitializeSListHead@4 1007e028     kernel32:KERNEL32.dll
 0002:0000002c       __imp__IsDebuggerPresent@0 1007e02c     kernel32:KERNEL32.dll
 0002:00000030       \177KERNEL32_NULL_THUNK_DATA 1007e030     kernel32:KERNEL32.dll
 0002:00000034       __imp__memcpy              1007e034     vcruntime:VCRUNTIME140.dll
 0002:00000038       __imp__memset              1007e038     vcruntime:VCRUNTIME140.dll
 0002:0000003c       __imp____std_type_info_destroy_list 1007e03c     vcruntime:VCRUNTIME140.dll
 0002:00000040       __imp___except_handler4_common 1007e040     vcruntime:VCRUNTIME140.dll
 0002:00000044       \177VCRUNTIME140_NULL_THUNK_DATA 1007e044     vcruntime:VCRUNTIME140.dll
 0002:00000048       __imp__malloc              1007e048     ucrt:api-ms-win-crt-heap-l1-1-0.dll
 0002:0000004c       __imp__free                1007e04c     ucrt:api-ms-win-crt-heap-l1-1-0.dll
 0002:00000050       \177api-ms-win-crt-heap-l1-1-0_NULL_THUNK_DATA 1007e050     ucrt:api-ms-win-crt-heap-l1-1-0.dll
 0002:00000054       __imp___seh_filter_dll     1007e054     ucrt:api-ms-win-crt-runtime-l1-1-0.dll
 0002:00000058       __imp___configure_narrow_argv 1007e058     ucrt:api-ms-win-crt-runtime-l1-1-0.dll
 0002:0000005c       __imp___initterm_e         1007e05c     ucrt:api-ms-win-crt-runtime-l1-1-0.dll
 0002:00000060       __imp___initialize_onexit_table 1007e060     ucrt:api-ms-win-crt-runtime-l1-1-0.dll
 0002:00000064       __imp___execute_onexit_table 1007e064     ucrt:api-ms-win-crt-runtime-l1-1-0.dll
 0002:00000068       __imp___cexit              1007e068     ucrt:api-ms-win-crt-runtime-l1-1-0.dll
 0002:0000006c       __imp___initterm           1007e06c     ucrt:api-ms-win-crt-runtime-l1-1-0.dll
 0002:00000070       __imp___initialize_narrow_environment 1007e070     ucrt:api-ms-win-crt-runtime-l1-1-0.dll
 0002:00000074       \177api-ms-win-crt-runtime-l1-1-0_NULL_THUNK_DATA 1007e074     ucrt:api-ms-win-crt-runtime-l1-1-0.dll
 0002:00000078       ___guard_check_icall_fptr  1007e078     MSVCRT:guard_support.obj
 0002:0000007c       ___castguard_check_failure_os_handled_fptr 1007e07c     MSVCRT:guard_support.obj
 0002:00000080       ___xc_a                    1007e080     MSVCRT:initializers.obj
 0002:00000084       ___xc_z                    1007e084     MSVCRT:initializers.obj
 0002:00000088       ___xi_a                    1007e088     MSVCRT:initializers.obj
 0002:0000008c       ___xi_z                    1007e08c     MSVCRT:initializers.obj
 0002:00000090       ___xp_a                    1007e090     MSVCRT:initializers.obj
 0002:00000094       ___xp_z                    1007e094     MSVCRT:initializers.obj
 0002:00000098       ___xt_a                    1007e098     MSVCRT:initializers.obj
 0002:0000009c       ___xt_z                    1007e09c     MSVCRT:initializers.obj
 0002:000000a0       _mlib_AffineFunArr_nn      1007e0a0     mlib_ImageAffine.obj
 0002:000000e0       _mlib_AffineFunArr_bl      1007e0e0     mlib_ImageAffine.obj
 0002:00000140       _mlib_AffineFunArr_bc      1007e140     mlib_ImageAffine.obj
 0002:000001a0       _mlib_AffineFunArr_bc_i    1007e1a0     mlib_ImageAffine.obj
 0002:000001c0       __real@3ef0000000000000    1007e1c0     mlib_ImageAffineEdge.obj
 0002:000001c8       __real@3fe0000000000000    1007e1c8     mlib_ImageAffineEdge.obj
 0002:000001d0       __real@3ff0000000000000    1007e1d0     mlib_ImageAffineEdge.obj
 0002:000001d8       __real@4004000000000000    1007e1d8     mlib_ImageAffineEdge.obj
 0002:000001e0       __real@4008000000000000    1007e1e0     mlib_ImageAffineEdge.obj
 0002:000001e8       __real@41dfe00000000000    1007e1e8     mlib_ImageAffineEdge.obj
 0002:000001f0       __real@41dfffe000000000    1007e1f0     mlib_ImageAffineEdge.obj
 0002:000001f8       __real@41dfffffffc00000    1007e1f8     mlib_ImageAffineEdge.obj
 0002:00000200       __real@c1e0000000000000    1007e200     mlib_ImageAffineEdge.obj
 0002:00000208       __real@37800000            1007e208     mlib_ImageAffine_BC_F32.obj
 0002:0000020c       __real@3f000000            1007e20c     mlib_ImageAffine_BC_F32.obj
 0002:00000210       __real@3f800000            1007e210     mlib_ImageAffine_BC_F32.obj
 0002:00000214       __real@40200000            1007e214     mlib_ImageAffine_BC_F32.obj
 0002:00000218       __real@40400000            1007e218     mlib_ImageAffine_BC_F32.obj
 0002:00000220       __real@bfc0000000000000    1007e220     mlib_ImageColorTrue2Index.obj
 0002:00000230       __xmm@00000004000000040000000400000004 1007e230     mlib_ImageColorTrue2Index.obj
 0002:00000240       __xmm@00000008000000080000000800000008 1007e240     mlib_ImageColorTrue2Index.obj
 0002:00000250       __xmm@ffffffffffffffffffffffffffffffff 1007e250     mlib_ImageColorTrue2Index.obj
 0002:00000260       __real@3e10000000000000    1007e260     mlib_ImageConv2x2_f.obj
 0002:00000268       __real@40f0000000000000    1007e268     mlib_ImageConv2x2_f.obj
 0002:00000270       __real@4170000000000000    1007e270     mlib_ImageConv2x2_f.obj
 0002:00000278       __real@41e0000000000000    1007e278     mlib_ImageConv2x2_f.obj
 0002:00000280       __real@41d0000000000000    1007e280     mlib_ImageConvKernelConvert.obj
 0002:00000290       __xmm@41dfffffffc0000041dfffffffc00000 1007e290     mlib_ImageConvKernelConvert.obj
 0002:000002a0       __xmm@41f00000000000000000000000000000 1007e2a0     mlib_ImageConvKernelConvert.obj
 0002:000002b0       __xmm@7fffffffffffffff7fffffffffffffff 1007e2b0     mlib_ImageConvKernelConvert.obj
 0002:000002c0       __xmm@c1e0000000000000c1e0000000000000 1007e2c0     mlib_ImageConvKernelConvert.obj
 0002:000002d0       __real@3f10000000000000    1007e2d0     mlib_ImageConv_16ext.obj
 0002:000002e0       __xmm@00000003000000020000000100000000 1007e2e0     mlib_ImageConv_16ext.obj
 0002:000002f0       __real@3f90000000000000    1007e2f0     mlib_ImageConv_8ext.obj
 0002:000002f8       _mlib_div6_tab             1007e2f8     mlib_ImageDivTables.obj
 0002:000004f8       _mlib_div1_tab             1007e4f8     mlib_ImageDivTables.obj
 0002:000006f8       _mlib_HSL2RGB_L2           1007e6f8     mlib_ImageDivTables.obj
 0002:00000af8       _mlib_HSL2RGB_F            1007eaf8     mlib_ImageDivTables.obj
 0002:00000ef8       _mlib_U82F32               1007eef8     mlib_ImageDivTables.obj
 0002:00001300       _mlib_U82D64               1007f300     mlib_ImageDivTables.obj
 0002:00001b08       _mlib_FlipAndFixRotateTable 1007fb08     mlib_ImageDivTables.obj
 0002:00002308       _mlib_filters_u8f_bc       10080308     mlib_ImageFilters.obj
 0002:00003308       _mlib_filters_u8f_bc2      10081308     mlib_ImageFilters.obj
 0002:00004308       _mlib_filters_s16f_bc      10082308     mlib_ImageFilters.obj
 0002:00006308       _mlib_filters_s16f_bc2     10084308     mlib_ImageFilters.obj
 0002:00008308       _mlib_filters_u8_bc        10086308     mlib_ImageFilters.obj
 0002:00008b08       _mlib_filters_u8_bc2       10086b08     mlib_ImageFilters.obj
 0002:00009308       _mlib_filters_s16_bc       10087308     mlib_ImageFilters.obj
 0002:0000a308       _mlib_filters_s16_bc2      10088308     mlib_ImageFilters.obj
 0002:0000b310       __xmm@00040000000400000004000000040000 10089310     mlib_ImageLookUp_64.obj
 0002:0000b320       __xmm@fffffff8fffffff8fffffff8fffffff8 10089320     mlib_ImageLookUp_64.obj
 0002:0000b3b0       __real@0000000000000000    100893b0     mlib_ImageScanPoly.obj
 0002:0000b3b8       __real@7fefffffffffffff    100893b8     mlib_ImageScanPoly.obj
 0002:0000b3c0       __real@bfe0000000000000    100893c0     mlib_ImageScanPoly.obj
 0002:0000b3c8       __real@ffefffffffffffff    100893c8     mlib_ImageScanPoly.obj
 0002:0000b3d0       __xmm@80000000000000008000000000000000 100893d0     mlib_ImageScanPoly.obj
 0002:0000b3e0       __real@4330000000000000    100893e0     mlib_ImageUtils.obj
 0002:0000b3e8       _mlib_AffineFunArr_bl_i    100893e8     mlib_c_ImageAffineIndex_BL.obj
 0002:0000b408       __real@4020000000000000    10089408     mlib_c_ImageConvVersion.obj
 0002:0000b410       __real@4040000000000000    10089410     mlib_c_ImageConvVersion.obj
 0002:0000b418       __real@40e0000000000000    10089418     mlib_c_ImageConvVersion.obj
 0002:0000b420       __xmm@00008000000080000000800000008000 10089420     mlib_c_ImageLookUp_f.obj
 0002:0000b430       __xmm@00010000000100000001000000010000 10089430     mlib_c_ImageLookUp_f.obj
 0002:0000b440       __xmm@00020000000200000002000000020000 10089440     mlib_c_ImageLookUp_f.obj
 0002:0000b450       __xmm@1fffffff1fffffff1fffffff1fffffff 10089450     mlib_c_ImageLookUp_f.obj
 0002:0000b460       __xmm@3ffffffe3ffffffe3ffffffe3ffffffe 10089460     mlib_c_ImageLookUp_f.obj
 0002:0000b470       __xmm@7ffffffc7ffffffc7ffffffc7ffffffc 10089470     mlib_c_ImageLookUp_f.obj
 0002:0000b480       __pDefaultRawDllMain       10089480     MSVCRT:dll_dllmain.obj
 0002:0000b480       __pRawDllMain              10089480     MSVCRT:dll_dllmain.obj
 0002:0000b490       __load_config_used         10089490     MSVCRT:loadcfg.obj
 0002:0000b5c0       ___safe_se_handler_table   100895c0     <linker-defined>
 0002:0000b5c4       ___volatile_metadata       100895c4     <linker-defined>
 0002:0000b92c       ___rtc_iaa                 1008992c     MSVCRT:initsect.obj
 0002:0000b930       ___rtc_izz                 10089930     MSVCRT:initsect.obj
 0002:0000b934       ___rtc_taa                 10089934     MSVCRT:initsect.obj
 0002:0000b938       ___rtc_tzz                 10089938     MSVCRT:initsect.obj
 0002:0000baf4       __IMPORT_DESCRIPTOR_KERNEL32 10089af4     kernel32:KERNEL32.dll
 0002:0000bb08       __IMPORT_DESCRIPTOR_VCRUNTIME140 10089b08     vcruntime:VCRUNTIME140.dll
 0002:0000bb1c       __IMPORT_DESCRIPTOR_api-ms-win-crt-heap-l1-1-0 10089b1c     ucrt:api-ms-win-crt-heap-l1-1-0.dll
 0002:0000bb30       __IMPORT_DESCRIPTOR_api-ms-win-crt-runtime-l1-1-0 10089b30     ucrt:api-ms-win-crt-runtime-l1-1-0.dll
 0002:0000bb44       __NULL_IMPORT_DESCRIPTOR   10089b44     kernel32:KERNEL32.dll
 0003:000002c0       ___security_cookie_complement 1008a2c0     MSVCRT:gs_cookie.obj
 0003:000002c4       ___security_cookie         1008a2c4     MSVCRT:gs_cookie.obj
 0003:000002c8       __fltused                  1008a2c8     MSVCRT:fltused.obj
 0003:000002d0       ___isa_enabled             1008a2d0     MSVCRT:cpu_disp.obj
 0003:000002e0       ___scrt_native_dllmain_reason 1008a2e0     MSVCRT:utility.obj
 0003:000002f0       ___scrt_ucrt_dll_is_in_use 1008a2f0     MSVCRT:ucrt_stubs.obj
 0003:000002f8       ___isa_available           1008a2f8     MSVCRT:cpu_disp.obj
 0003:000002fc       ___favor                   1008a2fc     MSVCRT:cpu_disp.obj
 0003:00000628       ?__type_info_root_node@@3U__type_info_node@@A 1008a628     MSVCRT:tncleanup.obj
 0003:00000630       ?_OptionsStorage@?1??__local_stdio_printf_options@@9@4_KA 1008a630     MSVCRT:default_local_stdio_options.obj
 0003:00000638       ?_OptionsStorage@?1??__local_stdio_scanf_options@@9@4_KA 1008a638     MSVCRT:default_local_stdio_options.obj
 0003:00000640       ___scrt_current_native_startup_state 1008a640     MSVCRT:utility.obj
 0003:00000644       ___scrt_native_startup_lock 1008a644     MSVCRT:utility.obj
 0003:00000664       ___scrt_debugger_hook_flag 1008a664     MSVCRT:utility_desktop.obj
 0003:00000668       ___dyn_tls_init_callback   1008a668     <common>

 entry point at        0001:0007ba6f

 Static symbols

 0000:fff72000       .debug$S                   10000000     mlib_image.exp
 0000:fff72000       .debug$S                   10000000     vcruntime:VCRUNTIME140.dll
 0000:fff72000       .debug$S                   10000000     vcruntime:VCRUNTIME140.dll
 0000:fff72000       .debug$S                   10000000     vcruntime:VCRUNTIME140.dll
 0000:fff72000       .debug$S                   10000000     vcruntime:VCRUNTIME140.dll
 0000:fff72000       .debug$S                   10000000     vcruntime:VCRUNTIME140.dll
 0000:fff72000       .debug$S                   10000000     vcruntime:VCRUNTIME140.dll
 0000:fff72000       .debug$S                   10000000     vcruntime:VCRUNTIME140.dll
 0000:fff72000       .debug$S                   10000000     ucrt:api-ms-win-crt-heap-l1-1-0.dll
 0000:fff72000       .debug$S                   10000000     ucrt:api-ms-win-crt-heap-l1-1-0.dll
 0000:fff72000       .debug$S                   10000000     ucrt:api-ms-win-crt-heap-l1-1-0.dll
 0000:fff72000       .debug$S                   10000000     ucrt:api-ms-win-crt-math-l1-1-0.dll
 0000:fff72000       .debug$S                   10000000     ucrt:api-ms-win-crt-math-l1-1-0.dll
 0002:fff82000       .idata$6                   10000000     ucrt:api-ms-win-crt-math-l1-1-0.dll
 0000:fff72000       .debug$S                   10000000     ucrt:api-ms-win-crt-runtime-l1-1-0.dll
 0000:fff72000       .debug$S                   10000000     ucrt:api-ms-win-crt-runtime-l1-1-0.dll
 0000:fff72000       .debug$S                   10000000     ucrt:api-ms-win-crt-runtime-l1-1-0.dll
 0000:fff72000       .debug$S                   10000000     ucrt:api-ms-win-crt-runtime-l1-1-0.dll
 0000:fff72000       .debug$S                   10000000     ucrt:api-ms-win-crt-runtime-l1-1-0.dll
 0000:fff72000       .debug$S                   10000000     ucrt:api-ms-win-crt-runtime-l1-1-0.dll
 0000:fff72000       .debug$S                   10000000     ucrt:api-ms-win-crt-runtime-l1-1-0.dll
 0000:fff72000       .debug$S                   10000000     ucrt:api-ms-win-crt-runtime-l1-1-0.dll
 0000:fff72000       .debug$S                   10000000     ucrt:api-ms-win-crt-runtime-l1-1-0.dll
 0000:fff72000       .debug$S                   10000000     ucrt:api-ms-win-crt-runtime-l1-1-0.dll
 0000:fff72000       .debug$S                   10000000     ucrt:api-ms-win-crt-runtime-l1-1-0.dll
 0000:fff72000       .debug$S                   10000000     ucrt:api-ms-win-crt-runtime-l1-1-0.dll
 0000:fff72000       .debug$S                   10000000     kernel32:KERNEL32.dll
 0000:fff72000       .debug$S                   10000000     kernel32:KERNEL32.dll
 0000:fff72000       .debug$S                   10000000     kernel32:KERNEL32.dll
 0000:fff72000       .debug$S                   10000000     kernel32:KERNEL32.dll
 0000:fff72000       .debug$S                   10000000     kernel32:KERNEL32.dll
 0000:fff72000       .debug$S                   10000000     kernel32:KERNEL32.dll
 0000:fff72000       .debug$S                   10000000     kernel32:KERNEL32.dll
 0000:fff72000       .debug$S                   10000000     kernel32:KERNEL32.dll
 0000:fff72000       .debug$S                   10000000     kernel32:KERNEL32.dll
 0000:fff72000       .debug$S                   10000000     kernel32:KERNEL32.dll
 0000:fff72000       .debug$S                   10000000     kernel32:KERNEL32.dll
 0000:fff72000       .debug$S                   10000000     kernel32:KERNEL32.dll
 0000:fff72000       .debug$S                   10000000     kernel32:KERNEL32.dll
 0000:fff72000       .debug$S                   10000000     kernel32:KERNEL32.dll
 0001:000003a8       $LN69                      100013a8     mlib_ImageAffine.obj
 0001:000003b8       $LN70                      100013b8     mlib_ImageAffine.obj
 0001:00010510       $LN1307                    10011510     mlib_ImageAffineEdge.obj
 0001:000159d0       $LN943                     100169d0     mlib_ImageAffineEdge.obj
 0001:00016d3c       $LN436                     10017d3c     mlib_ImageAffineEdge.obj
 0001:00017614       $LN245                     10018614     mlib_ImageAffineEdge.obj
 0001:00027ad0       $LN501                     10028ad0     mlib_ImageColorTrue2Index.obj
 0001:00027ae0       $LN503                     10028ae0     mlib_ImageColorTrue2Index.obj
 0001:00027af0       $LN502                     10028af0     mlib_ImageColorTrue2Index.obj
 0001:00027afc       $LN505                     10028afc     mlib_ImageColorTrue2Index.obj
 0001:00027b0c       $LN504                     10028b0c     mlib_ImageColorTrue2Index.obj
 0001:0002cf70       $LN842                     1002df70     mlib_ImageColorTrue2Index.obj
 0001:0002cf80       $LN843                     1002df80     mlib_ImageColorTrue2Index.obj
 0001:0002cfa0       $LN844                     1002dfa0     mlib_ImageColorTrue2Index.obj
 0001:0002d370       $LN70                      1002e370     mlib_ImageColorTrue2Index.obj
 0001:0002d380       $LN69                      1002e380     mlib_ImageColorTrue2Index.obj
 0001:0002d834       $LN74                      1002e834     mlib_ImageColorTrue2Index.obj
 0001:00030328       $LN511                     10031328     mlib_ImageColorTrue2Index.obj
 0001:00030338       $LN512                     10031338     mlib_ImageColorTrue2Index.obj
 0001:00030358       $LN513                     10031358     mlib_ImageColorTrue2Index.obj
 0001:00035058       $LN886                     10036058     mlib_ImageColorTrue2Index.obj
 0001:00035068       $LN887                     10036068     mlib_ImageColorTrue2Index.obj
 0001:00035088       $LN888                     10036088     mlib_ImageColorTrue2Index.obj
 0001:0003542c       $LN74                      1003642c     mlib_ImageColorTrue2Index.obj
 0001:00035914       $LN88                      10036914     mlib_ImageColorTrue2Index.obj
 0001:00038e54       $LN17                      10039e54     mlib_ImageConvMxN.obj
 0001:000393cc       $LN44                      1003a3cc     mlib_ImageConvMxN.obj
 0001:000393e4       $LN45                      1003a3e4     mlib_ImageConvMxN.obj
 0001:00039400       _mlib_ImageConvMxNMulAdd_D64 1003a400 f   mlib_ImageConvMxN_Fp.obj
 0001:000395f0       _mlib_ImageConvMxNMulAdd_F32 1003a5f0 f   mlib_ImageConvMxN_Fp.obj
 0001:0003a760       _mlib_ImageConv1xN_ext     1003b760 f   mlib_ImageConv_16ext.obj
 0001:0003f0b0       _mlib_ImageConv1xN         100400b0 f   mlib_ImageConv_16nw.obj
 0001:00042c00       _mlib_ImageConv1xN         10043c00 f   mlib_ImageConv_32nw.obj
 0001:00044f60       _mlib_ImageConv1xN_ext     10045f60 f   mlib_ImageConv_8ext.obj
 0001:000499d0       _mlib_ImageConv1xN         1004a9d0 f   mlib_ImageConv_8nw.obj
 0001:0004d400       _mlib_ImageConv1xN         1004e400 f   mlib_ImageConv_D64nw.obj
 0001:0004e9c0       _mlib_ImageConv1xN         1004f9c0 f   mlib_ImageConv_F32nw.obj
 0001:00050080       _mlib_ImageConv1xN_ext     10051080 f   mlib_ImageConv_u16ext.obj
 0001:00054b10       _mlib_ImageConv1xN         10055b10 f   mlib_ImageConv_u16nw.obj
 0001:00058c0c       $LN32                      10059c0c     mlib_ImageCreate.obj
 0001:00058e44       $LN32                      10059e44     mlib_ImageCreate.obj
 0001:00058f24       $LN18                      10059f24     mlib_ImageCreate.obj
 0001:00070e34       $LN216                     10071e34     mlib_c_ImageConvClearEdge.obj
 0001:00072128       $LN337                     10073128     mlib_c_ImageConvCopyEdge.obj
 0001:0007b4f0       $$000000                   1007c4f0     MSVCRT:chkstk.obj
 0001:0007b504       cs10                       1007c504     MSVCRT:chkstk.obj
 0001:0007b512       cs20                       1007c512     MSVCRT:chkstk.obj
 0001:0007b6f0       $$000000                   1007c6f0     MSVCRT:llshl.obj
 0001:0007b700       MORE32                     1007c700     MSVCRT:llshl.obj
 0001:0007b70a       RETZERO                    1007c70a     MSVCRT:llshl.obj
 0001:0007b710       $$000000                   1007c710     MSVCRT:ullshr.obj
 0001:0007b720       MORE32                     1007c720     MSVCRT:ullshr.obj
 0001:0007b72a       RETZERO                    1007c72a     MSVCRT:ullshr.obj
 0001:0007b72f       ?dllmain_crt_dispatch@@YGHQAUHINSTANCE__@@KQAX@Z 1007c72f f   MSVCRT:dll_dllmain.obj
 0001:0007b782       ?dllmain_crt_process_attach@@YAHQAUHINSTANCE__@@QAX@Z 1007c782 f   MSVCRT:dll_dllmain.obj
 0001:0007b889       ?dllmain_crt_process_detach@@YAH_N@Z 1007c889 f   MSVCRT:dll_dllmain.obj
 0001:0007b939       ?dllmain_dispatch@@YAHQAUHINSTANCE__@@KQAX@Z 1007c939 f   MSVCRT:dll_dllmain.obj
 0001:0007ba44       ?dllmain_raw@@YGHQAUHINSTANCE__@@KQAX@Z 1007ca44 f   MSVCRT:dll_dllmain.obj
 0001:0007bbb4       ___get_entropy             1007cbb4 f   MSVCRT:gs_support.obj
 0001:0007bcaf       ?find_pe_section@@YAPAU_IMAGE_SECTION_HEADER@@QAEI@Z 1007ccaf f   MSVCRT:utility.obj
 0001:0007c110       $$000000                   1007d110     MSVCRT:sehprolg4.obj
 0002:0000b330       _mlib_bit_mask             10089330     mlib_ImageLookUp_Bit.obj
 0002:0000b370       _mlib_bit_mask_2           10089370     mlib_ImageLookUp_Bit.obj
 0002:0000b380       _mlib_bit_mask_3           10089380     mlib_ImageLookUp_Bit.obj
 0002:0000b484       _GS_ExceptionPointers      10089484     MSVCRT:gs_report.obj
 0002:0000b940       __sehtable$?dllmain_crt_process_attach@@YAHQAUHINSTANCE__@@QAX@Z 10089940     MSVCRT:dll_dllmain.obj
 0002:0000b960       __sehtable$?dllmain_crt_process_detach@@YAH_N@Z 10089960     MSVCRT:dll_dllmain.obj
 0002:0000b988       __sehtable$?dllmain_dispatch@@YAHQAUHINSTANCE__@@KQAX@Z 10089988     MSVCRT:dll_dllmain.obj
 0002:0000b9a8       __sehtable$___scrt_is_nonwritable_in_current_image 100899a8     MSVCRT:utility.obj
 0002:0000b9d0       .edata                     100899d0     mlib_image.exp
 0002:0000b9f8       rgpv                       100899f8     mlib_image.exp
 0002:0000ba14       rgszName                   10089a14     mlib_image.exp
 0002:0000ba30       rgwOrd                     10089a30     mlib_image.exp
 0002:0000ba3e       szName                     10089a3e     mlib_image.exp
 0002:0000ba4d       $N00001                    10089a4d     mlib_image.exp
 0002:0000ba62       $N00002                    10089a62     mlib_image.exp
 0002:0000ba82       $N00003                    10089a82     mlib_image.exp
 0002:0000ba98       $N00004                    10089a98     mlib_image.exp
 0002:0000baad       $N00005                    10089aad     mlib_image.exp
 0002:0000bac8       $N00006                    10089ac8     mlib_image.exp
 0002:0000badd       $N00007                    10089add     mlib_image.exp
 0002:0000bcf4       .idata$6                   10089cf4     kernel32:KERNEL32.dll
 0002:0000bd50       .idata$6                   10089d50     vcruntime:VCRUNTIME140.dll
 0002:0000be1a       .idata$6                   10089e1a     ucrt:api-ms-win-crt-heap-l1-1-0.dll
 0002:0000be3a       .idata$6                   10089e3a     ucrt:api-ms-win-crt-runtime-l1-1-0.dll
 0003:00000000       ?opposite_quadrants@?1??mlib_search_quadrant_part_to_left_U8_3@@9@9 1008a000     mlib_ImageColorTrue2Index.obj
 0003:00000030       ?opposite_quadrants@?1??mlib_search_quadrant_part_to_right_U8_3@@9@9 1008a030     mlib_ImageColorTrue2Index.obj
 0003:00000060       ?opposite_quadrants@?1??mlib_search_quadrant_part_to_left_S16_3@@9@9 1008a060     mlib_ImageColorTrue2Index.obj
 0003:00000090       ?opposite_quadrants@?1??mlib_search_quadrant_part_to_right_S16_3@@9@9 1008a090     mlib_ImageColorTrue2Index.obj
 0003:000000c0       ?opposite_quadrants@?1??mlib_search_quadrant_part_to_left_U8_4@@9@9 1008a0c0     mlib_ImageColorTrue2Index.obj
 0003:00000140       ?opposite_quadrants@?1??mlib_search_quadrant_part_to_right_U8_4@@9@9 1008a140     mlib_ImageColorTrue2Index.obj
 0003:000001c0       ?opposite_quadrants@?1??mlib_search_quadrant_part_to_left_S16_4@@9@9 1008a1c0     mlib_ImageColorTrue2Index.obj
 0003:00000240       ?opposite_quadrants@?1??mlib_search_quadrant_part_to_right_S16_4@@9@9 1008a240     mlib_ImageColorTrue2Index.obj
 0003:00000300       ?__proc_attached@@3HA      1008a300     MSVCRT:dll_dllmain.obj
 0003:00000308       _GS_ExceptionRecord        1008a308     MSVCRT:gs_report.obj
 0003:00000358       _GS_ContextRecord          1008a358     MSVCRT:gs_report.obj
 0003:00000648       ?is_initialized_as_dll@@3_NA 1008a648     MSVCRT:utility.obj
 0003:00000649       ?module_local_atexit_table_initialized@@3_NA 1008a649     MSVCRT:utility.obj
 0003:0000064c       ?module_local_atexit_table@@3U_onexit_table_t@@A 1008a64c     MSVCRT:utility.obj
 0003:00000658       ?module_local_at_quick_exit_table@@3U_onexit_table_t@@A 1008a658     MSVCRT:utility.obj
 0004:00000060       $R000000                   1008b060     mlib_image.dll.res
